:020000040800F2
:10000000000001201D210008551F0008571F00088F
:10001000591F00085B1F00085D1F0008000000005A
:100020000000000000000000000000005F1F00084A
:10003000611F000800000000631F0008651F000822
:100040006521000865210008652100086521000878
:100050006521000865210008652100086521000868
:100060006521000865210008652100086521000858
:100070006521000865210008691F0008751F000838
:100080006521000865210008652100086521000838
:100090006521000865210008652100086521000828
:1000A0006521000865210008652100086521000818
:1000B0006521000865210008652100086521000808
:1000C00065210008652100086521000865210008F8
:1000D00065210008811F00086521000865210008CE
:1000E00065210008652100086521000865210008D8
:1000F00065210008652100086521000865210008C8
:1001000065210008652100086521000865210008B7
:1001100065210008652100088D1F00086521000881
:100120006521000865210008652100086521000897
:1001300000000000000000000000000000000000BF
:1001400000000000000000000000000000000000AF
:10015000000000000000000000000000000000009F
:10016000000000000000000000000000000000008F
:10017000000000000000000000000000000000007F
:10018000000000000000000000000000000000006F
:10019000000000000000000000000000000000005F
:1001A000000000000000000000000000000000004F
:1001B000000000000000000000000000000000003F
:1001C000000000000000000000000000000000002F
:1001D000000000000000000000000000000000001F
:0401E0005FF8E0F1F3
:1001E40010B5054C237833B9044B13B10448AFF36D
:1001F40000800123237010BD800000200000000057
:100204001832000808B5034B1BB103490348AFF388
:10021400008008BD0000000084000020183200089F
:10022400D0400B1CD1409C46203AD3401843524244
:10023400634693401843704738B50E4B054618780B
:100244004FF47A73B3FBF0F30B4A1068B0FBF3F08E
:1002540000F08CF8044658B90F2D09D802462946F7
:100264004FF0FF3000F042F8044B20461D6038BDCB
:10027400012038BD000000201800002004000020E8
:10028400074A08B51368032043F01003136000F015
:100294001BF80020FFF7D0FF01F0B8FD002008BDD7
:1002A40000200240034A044B11681B780B4413607E
:1002B400704700BFD004002000000020014B1868E4
:1002C400704700BFD0040020074A0002D36800F43E
:1002D400E06023F4E0631B041B0C43F0BF6343F4AE
:1002E40000330343D360704700ED00E0174B30B593
:1002F400DC68C4F30224C4F10703251D042B28BFC2
:100304000423062D4FF0010598BF002405FA03F3DA
:1003140003F1FF3388BF033C1940A14005FA04F4FC
:10032400013C2240002842EA01024FEA0212AFBF18
:1003340000F16040064B00F00F00D2B2A5BFD2B26C
:1003440000F561401A5480F8002330BD00ED00E050
:1003540014ED00E00123420900F01F0003FA00F04D
:10036400014B43F82200704700E100E00138B0F18E
:10037400807F0AD2F021064B064A586082F8231087
:100384000020072298601A6070470120704700BF60
:1003940010E000E000ED00E010B5002832D0016864
:1003A400194B1424994225D8184AA3F207430A4446
:1003B400B2FBF4F2920002648468C36343680A687F
:1003C4002343C46822F47F522343046922F0300299
:1003D40023434469234384692343C4692343134364
:1003E4000B600122002380F82120836380F82030F1
:1003F400184610BD064B0B44B3FBF4F39B00036497
:10040400044BD9E7012010BD07040240F8FFFDBFEB
:10041400F8FBFDBF00040240F0B590F82040012C29
:1004240035D0012490F8215080F82040A5424FF0A7
:1004340000064FF0020428D180F821400468866346
:100444002668076C26F001062660C66BBD40756001
:10045400636043680568102BC36A0BBFA260A16088
:10046400E160E2604BB1236843F00E0323602B6824
:10047400002043F001032B60F0BD236823F0040344
:100484002360236843F00A03F0E780F82060022029
:10049400F0BD000090F8213010B5022B03D00423E6
:1004A4008363012010BD03681A6822F00E021A60EB
:1004B4001A6822F001021A60294A934224D902F5EB
:1004C4006272934219D01432934218D01432934278
:1004D40017D0143293420CBF4FF480534FF480333F
:1004E400204A53600123002480F82130436B80F8B4
:1004F40020409BB39847204610BD0123F0E710230A
:10050400EEE74FF48073EBE717498B4216D01431B2
:100514008B4215D014318B4214D014318B4214D039
:1005240014318B4214D014318B4214D0934214BF33
:100534004FF480334FF080730C4AD2E70123FBE77A
:100544001023F9E74FF48073F6E74FF48053F3E791
:100554004FF48033F0E74FF48013EDE7184610BDF5
:1005640080000240000402400800024000000240F3
:1005740070B40425C66B026C346803689540254248
:10058400196855D04D0753D51A6896065EBF1A6888
:1005940022F004021A60604A93421FD902F5627283
:1005A400934214D01432934213D01432934212D093
:1005B400143293420CBF4FF480434FF48023574AC4
:1005C4005360C36A002B00F0A58070BC1847042355
:1005D400F5E74023F3E74FF48063F0E750498B429B
:1005E40016D014318B4215D014318B4214D01431EF
:1005F4008B4214D014318B4214D014318B4214D05A
:10060400934214BF4FF480234FF08063454AD7E7E9
:100614000423FBE74023F9E74FF48063F6E74FF444
:100624008043F3E74FF48023F0E74FF48003EDE7D2
:1006340002259540254257D08D0755D51A68940652
:1006440006D41A6822F00A021A60012280F82120D6
:10065400314A93421ED902F56272934213D0143286
:10066400934212D01432934211D0143293420CBFED
:100674004FF400534FF40033284A5360002380F8AA
:100684002030836A9EE70223F6E72023F4E74FF441
:100694000073F1E722498B4216D014318B4215D0F6
:1006A40014318B4214D014318B4214D014318B4248
:1006B40014D014318B4214D0934214BF4FF400333E
:1006C4004FF00073174AD8E70223FBE72023F9E72A
:1006D4004FF40073F6E74FF40053F3E74FF400339D
:1006E400F0E74FF40013EDE708259540254211D0BB
:1006F40009070FD5196821F00E011960012303FAC7
:1007040002F27260836380F82130002380F8203085
:10071400036B57E770BC704780000240000402403E
:100724000800024000000240114AD36813F010038D
:1007340005D01049CB6943F00203CB611023D26882
:10074400500706D50B4943F00403CA6942F001027D
:10075400CA61074AD169C90708D50648C16941F089
:100764000401C161D16921F00101D161D3607047F5
:1007740000200240D8040020064B186910F08000C5
:1007840007D0054A5A6002F188325A601869C0F3EA
:10079400C01070470020024023016745034A00202F
:1007A400136943F080031361704700BF00200240C7
:1007B400F8B50646FFF782FD114C07462546E36867
:1007C400D80712D4E368990644BF2023E360EB689A
:1007D400DA0606D4EB69DB0703D4E86810F00400FA
:1007E40002D0FFF7A1FF0120F8BD731CE7D00EB9BA
:1007F4000320F8BDFFF762FDC01B8642DFD2F7E796
:10080400002002402DE9F84F1F4C9946237E0546EF
:10081400012B0F46904633D001234CF250302376FF
:10082400FFF7C6FF40BB012D03D0022D0CBF0225EC
:1008340004250026B246DFF854B03201404649464A
:10084400FFF7EEFCC4F81CA0DBF8103080B243F0D4
:100854000103CBF8103027F816004CF25030FFF7A4
:10086400A7FFDBF8103023F00103CBF8103018B9E0
:100874000136F3B29D42E0D800232376BDE8F88F19
:100884000220BDE8F88F00BFD804002000200240F9
:100894000022064BDA61064B1A6942F004021A611F
:1008A4001A6942F040021A61704700BFD804002060
:1008B400002002400022064BDA61064B1A6942F01E
:1008C40002021A6158611A6942F040021A617047C3
:1008D400D8040020002002402DE9F041234D0746B2
:1008E4002B7E8846012B3DD0012403682C76022BF5
:1008F4004CF2503013D1FFF75BFF20B101200023ED
:100904002B76BDE8F081FFF7C3FF4CF25030FFF7C0
:100914004FFF174A136923F004031361EFE7FFF74E
:1009240047FF0028EAD14FF0FF33C8F800302046D3
:10093400BE680F4CFA68BB6803EBC2239E42DED24A
:100944003046FFF7B7FF4CF25030FFF731FF236911
:1009540023F00203236110B1C8F80060CFE706F565
:100964000066E7E70220BDE8F08100BFD80400205C
:10097400002002402DE9F74F002216466C4F6D4BC4
:10098400DFF8B8E1DFF8B8C14FF001080C6808FAE5
:1009940006F808EA0404A04540F085804D68122D4D
:1009A40000F0B78000F28D80022D00F0AF8000F2DD
:1009B4008180002D00F09180012D00F0A5804FF082
:1009C4000F09FF2C93BF824606F18045083DD0F8FD
:1009D40000B092BFB500D0F804B0AD0009FA05F834
:1009E4002BEA080802FA05F588BF00F1040A48EA70
:1009F4000505CAF80050D1F804A01AF0805F52D05F
:100A0400BD6926F0030845F00105BD61BD6908F123
:100A1400804805F00105019508F5803806F0030BC0
:100A2400019D4FEA8B0BD8F8085009FA0BF925EA17
:100A34000909414DA84271D005F58065A8426FD0DF
:100A440005F58065A8426DD005F58065A8426BD098
:100A540005F58065A84269D070450CBF05250625BB
:100A640005FA0BF545EA0905C8F808501D681AF49B
:100A7400803F14BF2543A5431D605D681AF4003F01
:100A840014BF2543A5435D609D681AF4801F14BFFD
:100A94002543A5439D60DD681AF4001F14BF2C4351
:100AA40025EA0404DC600136102E7FF46DAF03B038
:100AB400BDE8F08F032D25D0112D80D1CA680432F2
:100AC4007DE7654509D012D8DFF878904D4504D00C
:100AD40009F580394D457FF472AF8A68E2B1012A85
:100AE4000CBFC0F81080C0F81480082267E7DFF854
:100AF40058904D45F1D009F580394D45EDD0A9F513
:100B04008019E7E700225AE7CA6858E7CA6808323A
:100B140055E7CA680C3252E7042250E700259FE7E4
:100B240001259DE702259BE7032599E7042597E71F
:100B3400001002400004014000080140001C014074
:100B44000000211000001110000031100AB10161F1
:100B540070470904FBE7C3685940C160704700004F
:100B640003682DE9F341DB07054610D42B689F0782
:100B74005ED42B68190700F195802B685A0700F1A1
:100B8400BF80EA69002A40F02D81002014E0904CD7
:100B9400636803F00C03042B07D0636803F00C03B1
:100BA400082B0CD16368DE0309D523689C03DDD5CB
:100BB4006B68002BDAD1012002B0BDE8F0816B68CC
:100BC400B3F5803F10D1236843F480332360FFF7EB
:100BD40075FB064623689803C8D4FFF76FFB801B98
:100BE4006428F7D90320E7E79BB9236823F480330B
:100BF4002360236823F480232360FFF75FFB06460A
:100C040023689903B2D5FFF759FB801B6428F7D9F1
:100C1400E8E7B3F5A02F236803D143F480232360CE
:100C2400D1E723F480332360236823F48023CDE7C2
:100C3400674C636813F00C0F07D0636803F00C0370
:100C4400082B10D16368DA030DD423689B0702D5FF
:100C54002B69012BAFD123686A6923F0F80343EAB7
:100C6400C203236085E72A695A4B6AB101221A60DC
:100C7400FFF724FB064623689F07ECD4FFF71EFB0F
:100C8400801B0228F7D9ADE71A60FFF717FB064669
:100C9400236898077FF56DAFFFF710FB801B0228D0
:100CA400F6D99FE7AA694A4C4B4BDAB101221A6084
:100CB400FFF704FB0646636A9B070DD54FF4FA520F
:100CC400464B1B68B3FBF2F3019300BF019B5A1E12
:100CD4000192002BF9D150E7FFF7F0FA801B0228AC
:100CE400E9D97FE71A60FFF7E9FA0646636A9F07C6
:100CF4007FF543AFFFF7E2FA801B0228F6D971E7CC
:100D0400334CE369D80024D40127E36943F08053CA
:100D1400E361E36903F080530093009B304E336832
:100D2400D90518D5EB68012B26D1236A43F00103BA
:100D34002362FFF7C3FA41F288368046236A9B0791
:100D44003FD5002F3FF41DAFE36923F08053E361E7
:100D540017E70027E2E7336843F480733360FFF753
:100D6400ADFA80463368DA05DCD4FFF7A7FAA0EBC6
:100D740008006428F6D935E7ABB9236A41F288380C
:100D840023F001032362236A23F004032362FFF7A1
:100D940095FA0646236A9807D3D5FFF78FFA801B86
:100DA4004045F7D91EE7052B236A03D143F004031A
:100DB4002362BAE723F001032362236A23F00403C6
:100DC400B6E7FFF77BFAA0EB0800B042B6D909E713
:100DD40000100240000042428004424218000020F9
:100DE40000700040224C636803F00C03082B3FF4AE
:100DF400E2AE00231F4E022A33602BD1FFF75EFAC6
:100E04000746236899011FD42B6AB3F5803F05D1A7
:100E14006268A96822F400320A436260696A6268FF
:100E24000B4322F474121343636001233360FFF70E
:100E340045FA054623689A013FF5A7AEFFF73EFA47
:100E4400401B0228F6D9CDE6FFF738FAC01B02286A
:100E5400D7D9C7E6FFF732FA054623689B017FF529
:100E640094AEFFF72BFA401B0228F6D9BAE600BF6E
:100E7400001002406000424230B5194B87B002AC0A
:100E840003F11005224618685968083303C2AB42BF
:100E94001446F7D101238DF80430022311498DF84B
:100EA40005304B6803F00C02082A17D1C3F38342C0
:100EB40006A80244DB0312F8102C0CD54B680A4830
:100EC400C3F34043504306AA134413F8143CB0FB45
:100ED400F3F007B030BD05485043FAE70248F8E79D
:100EE400303200080010024000127A0000093D0070
:100EF400544A2DE9F0411368054603F007038B4279
:100F04000E462AD329688C0734D4CA0747D44D4ADD
:100F1400136803F007039E42C0F082802A684A4C9B
:100F240012F0040F40F08780130706D563682A691E
:100F340023F4605343EAC2036360FFF79DFF6368D1
:100F4400424AC3F30313D35CD840414B18600020DA
:100F5400FFF772F90020BDE8F081136823F007035E
:100F64000B431360136803F007039942CAD00120AE
:100F7400BDE8F081344B11F0040F1EBF5A6842F4EF
:100F8400E0625A60080742BF5A6842F460525A60ED
:100F94005A68A86822F0F00202435A60B5E76A680A
:100FA400294C012A23681CD113F4003FDFD0636865
:100FB40041F2883823F0030313436360FFF77EF99B
:100FC4006B680746012B14D1636803F00C03042BF0
:100FD4009DD0FFF773F9C01B4045F5D90320BDE848
:100FE400F081022A02D113F0007FDFE713F0020F31
:100FF400DCE7022B0FD1636803F00C03082B86D0C7
:10100400FFF75CF9C01B4045F5D9E7E7FFF756F950
:10101400C01B4045E2D8636813F00C0FF6D176E7A5
:10102400136823F0070333431360136803F00703C3
:101034009E429CD172E76368E96823F4E0630B4342
:10104400636071E700200240001002409B320008F8
:1010540018000020044B054A5B68C3F30223D35CE9
:10106400034A1068D840704700100240AB320008B1
:1010740018000020044B054A5B68C3F3C223D35C09
:10108400034A1068D840704700100240AB32000891
:101094001800002003680020DA6842F00102DA60D8
:1010A4001A6842F001021A6070477047704770472F
:1010B4007047036810B51A69044691070ED5DA68BB
:1010C40092070BD56FF002021A6101229B69027725
:1010D4009B0777D0FFF7EAFF0023237723681A6979
:1010E400500710D5DA6851070DD56FF004021A6164
:1010F40002229B69227713F4407F204668D0FFF7D1
:10110400D5FF0023237723681A6912070FD5DA68FD
:1011140010070CD56FF008021A610422DB692277EC
:10112400990720465AD0FFF7C1FF0023237723688D
:101134001A69D20610D5DA68D0060DD56FF0100200
:101144001A610822DB69227713F4407F20464BD0D2
:10115400FFF7ACFF0023237723681A69D10708D56A
:10116400DA68D20705D56FF0010220461A6100F053
:1011740027FD23681A69100608D5DA68110605D513
:101184006FF0800220461A6100F0BFF823681A69E4
:10119400520608D5DA68500605D56FF0400220469D
:1011A4001A61FFF785FF23681A69910622D5DA6868
:1011B40092061FD56FF020022046BDE810401A6148
:1011C40000F0A2B8FFF771FF2046FFF770FF83E736
:1011D400FFF76BFF2046FFF76AFF92E7FFF765FF13
:1011E4002046FFF764FFA0E7FFF75FFF2046FFF705
:1011F4005EFFAFE710BD0000244A0368904212D09E
:1012040002F5006290420ED0B0F1804F0BD0A2F5EF
:101214009832904207D002F58062904203D002F5E2
:10122400806290421DD14A6823F070031343174A29
:10123400904212D002F5006290420ED0B0F1804F7D
:101244000BD0A2F59832904207D002F5806290420A
:1012540003D002F58062904203D1CA6823F440733C
:1012640013434A6923F08003134303608B68C3620A
:101274000B688362054B984203D003F500639842E0
:1012840001D10B690363012343617047002C0140C2
:1012940010B50446A0B190F83D3003F0FF021BB92D
:1012A40080F83C2000F0D4FD0223206884F83D300F
:1012B400211DFFF7A1FF0123002084F83D3010BD5C
:1012C400012010BD90F83C3010B5012B4FF0020303
:1012D40018D080F83D3003680C685A68496822F0D9
:1012E40070025A605A6822435A609A6822F0800257
:1012F4009A609A680A439A60012380F83D3000237B
:1013040080F83C30184610BD704770470368DA68AF
:1013140022F49072DA605A6922F001025A612023A1
:1013240080F83A30704700002DE9F0470568C2683C
:101334002B69016923F4405313432B618368EA68E2
:101344000B43416922F4B05222F00C020B431343C5
:10135400EB606B69826923F4407313436B61404B08
:1013640081469D424FF0190446D1FFF783FE04FBEA
:1013740000F3D9F804604FF06408B600B3FBF6F349
:10138400B3FBF8F31E01FFF775FE6043D9F8043090
:101394009B00B0FBF3F7FFF76DFE6043D9F8043010
:1013A4009B00B0FBF3F3B3FBF8F308FB13731B01CF
:1013B4003233B3FBF8F303F0F007FFF75BFE60434F
:1013C400D9F804209200B0FBF2FAFFF753FE604311
:1013D400D9F804309B00B0FBF3F3B3FBF8F308FB3C
:1013E40013A31B013233B3FBF8F303F00F033B43A6
:1013F4003344AB60BDE8F087FFF72CFE04FB00F339
:10140400D9F804604FF06408B600B3FBF6F3B3FBFD
:10141400F8F31E01FFF71EFE6043D9F804309B0069
:10142400B0FBF3F7FFF716FE6043D9F804309B00D6
:10143400B0FBF3F3B3FBF8F308FB13731B01323374
:10144400B3FBF8F303F0F007FFF704FE6043D9F8A9
:1014540004209200B0FBF2FAFFF7FCFDB7E700BFEF
:1014640000380140F8B504460E4617461D4621686B
:101474000B6836EA030301D10020F8BD6B1CF7D0DA
:1014840095B923680320DA6822F4D072DA605A69C5
:1014940022F001025A61202384F8393084F83A306A
:1014A400002384F83830F8BDFEF708FFC01B8542DE
:1014B400DDD2E6E710B5044640B390F8393003F0C6
:1014C400FF021BB980F8382000F0D6FC24232268E0
:1014D40084F83930D368204623F40053D360FFF7EF
:1014E40023FF236800201A6922F490421A615A6982
:1014F40022F02A025A61DA6842F40052DA602023A8
:10150400E06384F8393084F83A3010BD012010BD0E
:101514002DE9F0411F4690F839300446202B0D4642
:1015240090464ED1002949D0002A47D090F838304F
:10153400012B46D0012380F838300023C3632123D4
:1015440080F83930FEF7BAFE0646A4F82480A4F8E1
:101554002680E38C9BB26BB93B4632464021204641
:10156400FFF780FFA8B9202384F8380084F83930C5
:10157400BDE8F081E38C3246013B9BB2E384A3686F
:101584008021B3F5805F20463B460ED1FFF76AFF0A
:1015940010B10320BDE8F0812B882268C3F308034F
:1015A4005360236943B90235D3E7FFF75BFF002893
:1015B400EFD123682A785A600135CAE70120BDE8D3
:1015C400F0810220BDE8F08138B50446134694F852
:1015D4003920202A2AD139B333B394F83820012A88
:1015E40024D00122002584F838202122E384206BB2
:1015F400E56384F839200E4AA384216282620D4A8D
:101604004563C2620C4A026322680432FEF704FF97
:101614006FF04002236828461A605A6984F83850EB
:1016240042F080025A6138BD012038BD022038BD25
:10163400D316000801170008CD170008134690F8C8
:101644003A2073B5202A054638D1002934D0002B1E
:1016540032D090F83820012A30D00122002480F8BA
:101664003820222281628385C46380F83A20406B4B
:10167400134A2E688262134A4463C262124A0263A6
:101684000A46311DFEF7C8FE20462B6801941A68ED
:1016940001925A6885F838400192019ADA6842F456
:1016A4008072DA605A6942F001025A615A6942F062
:1016B40040025A6102B070BD0120FBE70220F9E745
:1016C4000B170008C1170008CD170008704708B5AC
:1016D4000368426A1B6813F020030AD1D384136899
:1016E4005A6922F080025A61DA6842F04002DA60F4
:1016F40008BD1046FFF7EAFF08BD704708B5406A09
:10170400FFF7FBFF08BD08B50368426A1B6813F0C6
:10171400200310D1D3851368D96821F48071D9606E
:10172400596921F001015961596921F04001596158
:10173400202382F83A30104600F0C0FC08BD90F82F
:101744003A3010B5222B36D183680169B3F5805F36
:101754000268836A23D15268E9B9C2F3080223F804
:10176400022B8362C48D013CA4B2C4858CB9036886
:10177400DA6822F02002DA60DA6822F48072DA6031
:101784005A6922F001025A61202380F83A3000F0AD
:1017940095FC002010BDD2B223F8012BE1E721B95A
:1017A400591C526881621A70DCE75268591C8162C4
:1017B40002F07F02F7E7022010BD704708B5406AC7
:1017C400FFF7FBFF08BD7047416A08B50B685A690B
:1017D40091F8390021280AD1120608D50022CA84BA
:1017E400DA6822F0C002DA60202281F839205B69CD
:1017F40091F83A20222A06D15B0604D50023084634
:10180400CB85FFF783FDCB6B084643F01003CB6316
:10181400FFF7D9FF08BD0000036870B51A680446D5
:101824001607D9685D6907D196065AD58D0658D52D
:10183400BDE87040FFF783BF15F0010502D111F434
:10184400907F4ED0D30705D5CE0542BFE36B43F05E
:101854000103E363500704D51DB1E36B43F00203B6
:10186400E363930704D51DB1E36B43F00403E3631F
:10187400160704D51DB1E36B43F00803E363E36B80
:10188400002B66D0950604D5880602D52046FFF7BE
:1018940056FF236820465D69E26B110702D415F0F8
:1018A40040051AD0FFF732FD23685A69520610D555
:1018B4005A69606B22F040025A6150B1254B436370
:1018C400FEF7E8FD002844D0606BBDE87040436B30
:1018D40018472046FFF777FF70BDFFF774FFE563F5
:1018E40070BD160627D50D0625D594F83920212A72
:1018F4002FD1A268B2F5805F226A17D11188C1F393
:1019040008015960216979B902322262E28C013AF4
:1019140092B2E284EAB9DA6822F08002DA60DA6824
:1019240042F04002DA6070BD0132EEE7511C2162E0
:1019340012785A60EAE750060BD54A0609D5DA68E8
:10194400204622F04002DA60202384F83930FFF781
:10195400BDFE70BD5D19000808B50023406AC3854B
:10196400C384FFF730FF08BD10B5074CA178601C95
:1019740000F05EF8A178207103312046BDE81040E4
:10198400C9B200F0C1BB00BF0E00002070B5817861
:10199400044643185A78013000F065F8C0B20128B3
:1019A4000ED000231E4EA2785D1C0232DBB29A4296
:1019B4002FDA1C4800F07CFC22221B4B5A700FE0EB
:1019C4001122194D6A706278DD2A01D0EE2A07D1FE
:1019D400204600F0B9F8C0B2012801D122236B706F
:1019E400114DA978681C00F023F828716378EE2B58
:1019F40007D00A2B05D0A97828460331C9B200F0D4
:101A040083FB6378EE2B0AD1BDE87040074800F0F1
:101A14004FBCE15C304600F0D7FB2B46C3E770BDFA
:101A240040320008463200080800002057320008FF
:101A340010B5FF230446221AD2B2914201D81846A7
:101A440010BD14F8012B5340082213F0800F02F14B
:101A5400FF324FEA430318BF83F0310312F0FF0251
:101A6400DBB2F2D1E7E730B5FF2305462C1AE4B226
:101A7400A14203D89B1A5842584130BD15F8014B76
:101A84006340082413F0800F04F1FF344FEA43034A
:101A940018BF83F0310314F0FF04DBB2F2D1E5E7A1
:101AA400B0B50D4A00AFD3690C4823F01003D361DD
:101AB40000F0FEFB0A4B0B4A1B680B4C0B481360EF
:101AC400236000F0F5FB0A4B1B6883F30888236846
:101AD400BD46BDE8B04018470010024083320008FC
:101AE40004400008F8040020FC040020953200089B
:101AF400004000082DE9F041002407462646104D19
:101B0400DFF84080BB78023B9C4202DB3046BDE8F4
:101B1400F0813B19DA781B79296802EB032292B22F
:101B240000230120FEF76EFE18B1404600F0C0FB12
:101B340001262B68023402332B60E4B2E2E700BFD3
:101B44001400002068320008002373B5164D174CAA
:101B54002B60174B0646AB601F23EB60E36923F051
:101B64001003E361FEF708FE124B1A784AB901220A
:101B7400114928461A70FEF7AFFE10B10F4800F065
:101B840097FB3046FFF7B6FF0546FEF707FE2846EB
:101B9400E36943F01003E361E36903F01003019385
:101BA400019B02B070BD00BF9C00002000100240E9
:101BB40000400008B0000020AC000020743200088F
:101BC4000268084B9A420BD1074A13680133136029
:101BD400064A136801331360054A1368013313601E
:101BE400704700BF00100040BC000020B800002077
:101BF400B400002010B514460A230248FFF788FCFD
:101C0400204610BD8805002010B590B02822002180
:101C140006A800F0D1FA1422002101A800F0CCFAA1
:101C240001230A93102302240B934FF4501306A8A4
:101C34000F9306940D94FEF793FF0F234FF48062E5
:101C440001930023214601A802940393049205936F
:101C5400FFF74EF910B010BD80B588B0FEF710FB49
:101C6400FFF7D2FF10225C4D00210DEB020000F0C3
:101C7400A3FAAB69002243F00403AB61AB694FF4F0
:101C8400004103F004030293029BAB69534843F4FD
:101C94008073AB61AB69002403F480730393039BEB
:101CA400FEF754FF00224FF480414D48FEF74EFFEB
:101CB40001274FF40043022604A9484804930796D9
:101CC40005970694FEF756FE4FF4804304A9444852
:101CD4000493079605970694FEF74CFE6B694148FA
:101CE4003B436B616B69404A3B400193019B4FF45A
:101CF400E13380E80C000C2384604361C460046118
:101D04008461C461FFF7D6FB41F26F73374D3849E4
:101D1400284685E80A000923AC60EB60AC610494B2
:101D24000594FFF7B5FA04A9284604940594FFF72F
:101D3400C9FA224621460F20FEF7D8FA0F20FEF7F3
:101D440009FB224621462520FEF7D0FA2520FEF77E
:101D540001FB224621463620FEF7C8FA3620FEF75C
:101D6400F9FA224621460E20FEF7C0FA0E20FEF7AD
:101D7400F1FA2846FFF78EF91E4B21461B68184ED0
:101D8400986800F09DFAFFF7EFFD1B4800F05CF93E
:101D94001A4D1B4C2368B3F5FA7F06D94FF48041E2
:101DA4003046FEF7D8FE00232360134C0D4FA36882
:101DB400002B02DD2B681E2B03D8124F40F6B834DB
:101DC40005E0384600F04EF9F1E7FFF769FE3B689D
:101DD400A342FAD8DDE700BF00100240000801402A
:101DE400002001408805002000380140C80500207B
:101DF400001000401C00002008060020BC00002049
:101E0400B8000020B4000020704700000E4B82B0E0
:101E14009A6942F001029A619A6902F00102009201
:101E2400009ADA6942F08052DA61DB69074A03F00A
:101E340080530193019B536823F0E06343F0806374
:101E4400536002B0704700BF001002400000014020
:101E54000268084B82B09A420AD103F50033DA696A
:101E640042F01002DA61DB6903F010030193019B75
:101E740002B070470010004070B5064686B01022CC
:101E8400002102A800F098F932682B4B9A4251D1F4
:101E940003F558439A6902A942F480429A619A6907
:101EA400264802F480420092009A9A69002542F082
:101EB40004029A619B69224C03F004030193019B81
:101EC4004FF4007302930223039303230593FEF755
:101ED40051FD4FF48063194802A9029303950495B8
:101EE400FEF748FD174B204684E828008023A560B0
:101EF400E36025616561A561E561FEF74DFA08B10E
:101F0400FFF782FF4FF0100C0F4B746366620F4CA7
:101F1400802284E8081000232046A360E260236145
:101F24006361A361E361FEF737FA08B1FFF76CFF61
:101F34003463666206B070BD003801400008014099
:101F440044050020580002404400024000050020DF
:101F54007047FEE7FEE7FEE7FEE77047704770470D
:101F6400FEF7A0B90148FEF703BB00BF000500203F
:101F74000148FEF7FDBA00BF440500200148FFF701
:101F84004BBC00BF880500200148FFF792B800BF92
:101F9400C805002070B50E4615460C46A31B9D428D
:101FA40001DC284670BDAFF3008004F8010BF5E7AF
:101FB40008B50A4B0246196809B909491960694606
:101FC400186802448A4206D900F0CCF80C23036056
:101FD4004FF0FF3008BD1A6008BD00BFC0000020EC
:101FE400241600204FF0FF3070474FF400530020B8
:101FF4004B60704701207047002070470F4B1A68F0
:1020040042F001021A6059680D4A0A405A601A687F
:1020140022F0847222F480321A601A6822F4802238
:102024001A605A6822F4FE025A604FF41F029A6042
:102034004FF00062034B9A60704700BF00100240EB
:102044000000FFF800ED00E000230122436003607C
:10205400836002490248FFF7F1BA00BF140600206A
:1020640088050020114A38B51468631C1360104BAE
:10207400596803F10C000D5C0131B1F5006FA8BF84
:1020840000210C48596005559C680546013C9C603C
:102094005CB908481460FFF779FC23462B550134DA
:1020A400B4F5806FFAD1044A136038BDC40000202F
:1020B40008060020C8000020B4000020002310B54A
:1020C4000D4A0E4C136022680132B2F5006FB8BF9E
:1020D40013462360A3680133B3F5006FA36001DBEB
:1020E400FFF7C0FF236806490122BDE810401944E8
:1020F4000448FFF7A3BA00BFBC0000200806002074
:1021040014060020880500200A4601460148FFF70E
:102114005BBA00BF88050020002103E00B4B5B582D
:10212400435004310A480B4B42189A42F6D30A4AE8
:1021340002E0002342F8043B084B9A42F9D3FFF72C
:102144005DFF00F015F8FFF787FD70475433000872
:1021540000000020800000208000002024160020C1
:10216400FEE70000014B1868704700BF1C00002008
:1021740070B500250C4E0D4CA41BA410A54209D12A
:1021840001F048F800250A4E0A4CA41BA410A542ED
:1021940005D170BD56F8253098470135EEE756F85D
:1021A400253098470135F2E74C3300084C330008DA
:1021B4004C3300085033000803460244934200D1D4
:1021C400704703F8011BF9E70FB40A4B13B51C68F9
:1021D40024B1A36913B9204600F0DAFA05AB049AD6
:1021E400A1682046019300F09BFC02B0BDE81040BA
:1021F40004B070471C00002070B50E46054618B1A7
:1022040083690BB900F0C4FAAB69AC6813B928460A
:1022140000F0BEFA234B9C4217D16C68A3891B07BC
:102224001DD52369DBB1013EA36816F8011F013BEC
:10223400A360E9B9002B2EDA22460A21284600F0D1
:10224400F5F8013011D00A2070BD174B9C4201D122
:10225400AC68E3E7154B9C4208BFEC68DEE7214617
:10226400284600F035F90028DDD04FF0FF3070BD6E
:10227400002B04DAA269934206DB0A2904D02368FE
:102284005A1C22601970CFE72246284600F0CEF887
:102294000130C9D1E9E70A2023685A1C226018706A
:1022A40070BD00BFD8320008F8320008B832000808
:1022B400024B01461868FFF79FBF00BF1C000020B7
:1022C40000294FF480630CBF0222002200F000B802
:1022D4002DE9F7431D46514B04461E680F469046B0
:1022E40026B1B36913B9304600F052FA4C4B9C4204
:1022F40052D17468B8F1020F06D0B8F1010F00F2A0
:102304008980002DC0F286802146304600F0D6F93F
:10231400616B41B104F14403994202D0304600F0AC
:102324002DFB002363630023A3616360A3891B0661
:1023340003D52169304600F021FBA389B8F1020FCF
:1023440023F44A6323F00303A3815DD001AB6A46FF
:102354002146304600F0A6FAA3891843A0812DBB7C
:10236400009D284600F002FB074600284ED1DDF808
:102374000090A9453CD14FF0FF30A38943F00203FC
:10238400A3810023A36004F1470323602361012395
:10239400636103B0BDE8F083224B9C4201D1B46871
:1023A400A8E7214B9C4208BFF468A3E7002FD8D0CC
:1023B400B36913B9304600F0EBF9B8F1010F08BF67
:1023C400A389276004BF43F00103A381A389276184
:1023D40013F0080065611BD013F001004FF00003F7
:1023E4001FBF6D42A360A561184608BFA560D0E772
:1023F400484600F0BBFA07460028BCD0A3894D46E6
:1024040043F08003A381D3E70020B6E7A946F5E7AC
:10241400A060BEE74FF0FF30BBE700BF1C00002008
:10242400D8320008F8320008B8320008F8B50E4671
:102434001446054618B183690BB900F0A9F9214B7C
:102444009C422AD16C68A369A360A3891A072ED57C
:10245400236963B323692068F6B2C01A63693746F7
:10246400984204DB2146284600F028F928BBA368DB
:102474000130013BA36023685A1C22601E7063690B
:10248400984204D0A389DB0719D50A2E17D1214617
:10249400284600F013F990B10FE00B4B9C4201D198
:1024A400AC68D0E7094B9C4208BFEC68CBE72146F7
:1024B400284600F00DF80028CCD04FF0FF373846FE
:1024C400F8BD00BFD8320008F8320008B83200085E
:1024D400324B70B51D6806460C4625B1AB6913B97D
:1024E400284600F055F92E4B9C420FD16C68B4F984
:1024F4000C309AB215072CD4D00611D409223260BC
:1025040043F04003A3814FF0FF3070BD254B9C4244
:1025140001D1AC68EBE7244B9C4208BFEC68E6E7CA
:10252400510712D5616B41B104F14403994202D0C1
:10253400304600F023FA00236363A38923F02403C5
:10254400A3810023636023692360A38943F0080304
:10255400A38123694BB9A38903F42073B3F5007FE6
:1025640003D02146304600F0C1F9A28912F00103DC
:102574000CD00023A36063695B42A361236953B950
:10258400B4F90C3013F08000BAD170BD920758BF73
:102594006369A360F2E70020F7E700BF1C00002096
:1025A400D8320008F8320008B83200088A892DE9C8
:1025B400F041054610070C465AD44B68002B05DC45
:1025C4000B6C002B02DC0020BDE8F081E66A002ED3
:1025D400F9D0002312F480522F682B6033D0606D41
:1025E400A3895A0705D56368C01A636B0BB1236CC2
:1025F400C01A00230246E66A216A2846B047431CF3
:10260400A38906D129681D294BD82B4ACA40D6076D
:1026140047D5002262602269D904226004D5421C95
:1026240001D12B6803B96065616B2F600029CAD0A2
:1026340004F14403994202D0284600F09FF9002097
:102644006063BDE8F081216A01232846B047411C3C
:10265400C6D12B68002BC3D01D2B01D0162B01D162
:102664002F60B0E7A38943F04003A381BDE8F08164
:102674000F69002FA7D0930718BF00230E6808BF67
:102684004B69A6EB07080F608B60B8F1000F9ADD69
:1026940043463A46216A2846A66AB047002807DC22
:1026A400A38943F04003A3814FF0FF30BDE8F081DC
:1026B4000744A8EB0008E8E70100402038B50B699F
:1026C40005460C46DBB118B183690BB900F060F81C
:1026D4000C4B9C4209D16C68B4F90C307BB1214697
:1026E4002846BDE83840FFF761BF074B9C4201D143
:1026F400AC68F1E7054B9C4208BFEC68ECE70020AE
:1027040038BD00BFD8320008F8320008B8320008DB
:10271400014900F0A9B800BFC1260008002310B584
:10272400044603604360836081814366C281036120
:1027340043618361194608225C30FFF73DFD054B78
:1027440024626362044BA362044BE362044B23637D
:1027540010BD00BFA1300008C3300008FB300008E2
:102764001F31000870B568254A1E55430E4605F111
:10277400740100F04FF9044640B1002180E84200A2
:102784000C30A06005F16802FFF716FD204670BD0D
:10279400836910B5044633BB8364C3640365124B79
:1027A400124A1B688262984204BF0123836100F0CD
:1027B4001FF86060204600F01BF8A060204600F07F
:1027C40017F80022E06004216068FFF7A7FF0122E8
:1027D4000921A068FFF7A2FF02221221E068FFF797
:1027E4009DFF0123A36110BDB43200081527000822
:1027F400F8B51C4B07461E68B36913B93046FFF79A
:10280400C7FF4836B4687368013B03D5336833B1F6
:102814003668F7E7B4F90C506DB16834F4E7042175
:102824003846FFF79FFF30600028F1D10C2304469F
:102834003B602046F8BD4FF6FF73E38101236566D4
:10284400A3812560A560656025616561A561082295
:10285400294604F15C00FFF7AFFC6563A563A5643A
:10286400E564E6E7B43200082DE9F843804689467A
:10287400002600F1480414B93046BDE8F883A56881
:102884006768013F01D52468F5E7AB89012B07D9B7
:10289400B5F90E30013303D029464046C8470643F4
:1028A4006835EEE770B50E46B1F90E1090B0002908
:1028B40014461D4607DA00232B60B3891A0610D488
:1028C4004FF480630EE001AA00F04EFC0028F2DB16
:1028D400029A02F47042A2F500535A425A412A6005
:1028E400EEE740230020236010B070BD8B8973B5E0
:1028F4009D0706460C4607D504F147032360236170
:102904000123636102B070BD01AB6A46FFF7CAFFE1
:1029140000990546304600F07DF848B9B4F90C300A
:102924009A05EFD423F0030343F00203A381E3E702
:102934000D4BB362A389206043F08003A381009B05
:1029440020616361019B5BB1B4F90E10304600F065
:102954001DFC28B1A38923F0030343F00103A381E1
:10296400A3891D43A581CDE715270008024B014625
:10297400186800F04FB800BF1C00002038B50546A9
:10298400002943D051F8043C0C1F002BB8BFE418B5
:1029940000F02CFC1E4A1368104633B963601460BF
:1029A4002846BDE8384000F022BCA3420BD9216878
:1029B4006218934201BF1A685B6852182260636010
:1029C4000460EDE713465A680AB1A242FAD91968BD
:1029D4005818A0420BD1206801445818824219604B
:1029E400DED110685268014419605A60D8E702D9F0
:1029F4000C232B60D4E7206821188A4201BF116898
:102A040052680918216062605C60C9E738BD00BF84
:102A1400C804002070B5CD1C25F0030508350C2D25
:102A240038BF0C25002D064601DBA94203D90C232F
:102A34003360002070BD00F0D9FB234A146821469E
:102A440091B9224C23681BB9304600F017FB206073
:102A54002946304600F012FB431C26D10C23304695
:102A6400336000F0C4FBE4E70B685B1B1AD40B2B48
:102A74000FD90B60CC18CD50304600F0B8FB04F1F0
:102A84000B00231D20F00700C31A1BD05A42E2504A
:102A940070BD8C420BBF63684B681360636018BFE2
:102AA4000C46E9E70C464968CAE7C41C24F0030451
:102AB400A04205D0211A304600F0E0FA0130CDD012
:102AC4002560D9E770BD00BFC8040020CC040020F5
:102AD400936810B4013B002B936008DA9469A34215
:102AE40002DBCBB20A2B02D110BCFFF79FBC1368E8
:102AF400581C10601970C8B210BC7047F8B506466F
:102B04000F461446D518AC4201D1002007E03A46DE
:102B140014F8011B3046FFF7DBFF431CF3D1F8BD6B
:102B24002DE9F04F9DB00C4617460393064618B1A5
:102B340083690BB9FFF72CFE7C4B9C4257D1746818
:102B4400A38918075DD52369002B5AD00023099364
:102B540020238DF8293030234FF0010B8DF82A30D3
:102B6400B846454615F8013B002B55D1B8EB070A8A
:102B74000BD053463A4621463046FFF7BFFF01309B
:102B840000F0C480099B5344099398F80030002B4B
:102B940000F0BC8000234FF0FF32049307930592AA
:102BA40006938DF853301A9305222978604800F073
:102BB4000FFB05F10108049B002831D1D90644BF5D
:102BC40020228DF853201A0744BF2B228DF853205E
:102BD4002A782A2A2CD000210A20079AA84698F895
:102BE40000300135303B092B6DD971B326E0514BD0
:102BF4009C4201D1B468A3E74F4B9C4208BFF468E0
:102C04009EE721463046FFF763FC00289ED04FF034
:102C1400FF301DB0BDE8F08F252BA7D0A846A0E754
:102C2400434A4546801A0BFA00F018430490BBE768
:102C3400039A111D12680391002A01DB079204E034
:102C4400524243F002030792049398F800302E2B6B
:102C540010D198F8013008F101012A2B37D1039BD8
:102C640008F102081A1D1B680392002BB8BF4FF02D
:102C7400FF330593314D032298F80010284600F0E5
:102C8400A7FA40B14023401B03FA00F0049B08F16B
:102C940001080343049398F800100622284808F119
:102CA40001078DF8281000F093FA002834D0254B42
:102CB40003BB039B073323F0070308330393099BE8
:102CC4004B4409934CE700FB0232012186E70023C1
:102CD4000A2518460593884698F800200131303AB1
:102CE400092A03D9002BC5D00590C3E705FB0020B2
:102CF4000123F0E703AB00932246134B04A93046AB
:102D0400AFF30080B0F1FF3F8146D8D1A3895B06C1
:102D14003FF57DAF09987CE703AB009322460A4B4D
:102D240004A9304600F08AF8ECE700BFD832000866
:102D340018330008F8320008B83200081E330008BF
:102D44002233000800000000012B00082DE9F047A1
:102D540091461F468A680B6906469342B8BF1346DC
:102D6400C9F8003091F843200C46DDF8208012B1F8
:102D74000133C9F800302368990642BFD9F80030FE
:102D84000233C9F80030256815F0060507D104F1AF
:102D9400190AE368D9F800209B1A9D422ADB94F8AB
:102DA40043302268003318BF012392062FD404F164
:102DB400430239463046C047013022D02368E568D3
:102DC40003F00603042B18BF0025D9F800204FF0A8
:102DD400000908BFAD1AA368226908BF25EAE57592
:102DE4009342C4BF9B1AED181A344D451BD10020E1
:102DF400BDE8F0870123524639463046C0470130CA
:102E040003D14FF0FF30BDE8F0870135C1E7302032
:102E1400E11881F843005A1C94F845102244023307
:102E240082F84310C3E70123224639463046C0479F
:102E34000130E6D009F10109D7E700002DE9F0439C
:102E440017460A7E85B06E2A984606460C460C9BA9
:102E540001F1430E00F0BC801AD8632A2ED00AD8A0
:102E6400002A00F0C880582A00F08A8004F1420544
:102E740084F842202AE0642A01D0692AF6D1216824
:102E84001A6811F0800F23D0111D1960136827E010
:102E9400732A00F0B48008D86F2A2AD0702AE5D1AA
:102EA4000A6842F020020A6003E0752A21D0782AD9
:102EB400DCD178226F4984F8452064E01A6801F176
:102EC4004205111D1960136884F842300123A3E000
:102ED40011F0400F02F104011960D7D0B2F90030AB
:102EE400002B03DA2D225B4284F8432062490A2234
:102EF40017E02068196810F0800F03D0081D1860CF
:102F04000B6806E010F0400F01F104001860F7D0E0
:102F14000B886F2A14BF0A2208225749002084F81C
:102F240043006568002DA560C0F29C80206820F0F5
:102F340004002060002B3FD1002D40F095807546A1
:102F4400082A0BD12368DA0708D5236962689A42F4
:102F5400DEBF302305F8013C05F1FF35AEEB050378
:102F64002361CDF800803B4603AA21463046FFF793
:102F7400EDFE013055D14FF0FF3005B0BDE8F083D0
:102F840081F845203C492268186812F0800F00F14E
:102F940004051D6001D0036802E05506FBD50388D3
:102FA400D00744BF42F0200222601BB9226822F0FD
:102FB400200222601022B1E77546B3FBF2F002FB57
:102FC4001033CB5C05F8013D03460028F5D1B7E783
:102FD40008681A6810F0800F496904D0101D186041
:102FE4001368196007E010F0400F02F10400186044
:102FF4001368F6D01980002375462361B1E71A6877
:10300400111D1960156800216268284600F0E0F877
:1030140008B1401B606063682361002384F8433077
:103024009FE723692A4639463046C0470130A2D07B
:1030340023689B0707D5002504F11909E368039A5F
:103044009B1A9D4205DBE068039B9842B8BF184673
:1030540093E701234A4639463046C04701308AD0B7
:103064000135EBE7002BA7D10B7804F1420584F876
:10307400423065E73A3300082933000838B50023A5
:10308400054C054608462360FEF792FF431C02D117
:10309400236803B12B6038BD2016002010B50C4600
:1030A400B1F90E1000F0A4F80028ABBF636DA3893A
:1030B4001B1823F48053ACBF6365A38110BD2DE9B5
:1030C400F0411F468B890546DB050C46164605D59F
:1030D40002230022B1F90E1000F068F8A3893246E9
:1030E40023F48053A381B4F90E103B462846BDE86F
:1030F400F04100F017B810B50C46B1F90E1000F00D
:1031040055F8431CA38915BF606523F4805343F429
:103114008053A38118BFA38110BDB1F90E1000F034
:1031240013B8000038B50546084611460022054C80
:1031340022601A46FEF75EFD431C02D1236803B1E8
:103144002B6038BD2016002038B50023054C0546F9
:1031540008462360FEF746FF431C02D1236803B1EF
:103164002B6038BD2016002038B50023064C0546D8
:10317400084611462360FEF738FF431C02D123683A
:1031840003B12B6038BD00BF2016002038B50023E2
:10319400054C054608462360FEF72CFF431C02D16C
:1031A400236803B12B6038BD2016002038B50546CE
:1031B400084611460022054C22601A46FEF71CFF01
:1031C400431C02D1236803B12B6038BD20160020B4
:1031D40010B5C9B202449042034601D1002010BD8B
:1031E4001C7801308C42F6D1184610BD70477047E8
:1031F40038B50546084611460022054C22601A4699
:10320400FEF7C8FE431C02D1236803B12B6038BD0E
:1032140020160020F8B500BFF8BC08BC9E467047D5
:0C322400F8B500BFF8BC08BC9E4670471F
:1032300002030405060708090A0B0C0D0E0F1010F7
:10324000253032782000436865636B2053756D200C
:103250006572726F72200075706461746520436FCF
:103260006D706C657465200048414C204E4F5420B1
:103270004F4B20004572617365204661696C65643F
:10328000200D00626F6F74206C6F61646572207333
:1032900074617274006A756D702100000000000096
:1032A00000000001020304060708090000000001F5
:1032B00002030400200000200000000000000000C5
:1032C00000000000000000000000000000000000FE
:1032D00000000000000000000000000000000000EE
:1032E00000000000000000000000000000000000DE
:1032F00000000000000000000000000000000000CE
:1033000000000000000000000000000000000000BD
:103310000000000000000000232D302B2000686C0E
:103320004C006566674546470030313233343536E8
:103330003738394142434445460030313233343521
:0C3340003637383961626364656600004E
:04334C00090200086A
:04335000E50100088B
:103354000100000010000000BE11030500BEBE0BFA
:10336400030400EB0040000800A24A0420000020EF
:1033740000000000D8320008F8320008B832000813
:103384000000000000000000000000000000000039
:103394000000000000000000000000000000000029
:1033A4000000000000000000000000000000000019
:1033B4000000000000000000000000000000000009
:1033C40000000000000000000000000000000000F9
:040000050800211DB1
:00000001FF
